:1000000028EF00F0EA6A050EE96EEF500EE00F0EE1
:10001000016E006A002EFED7012EFBD78F0E006EF8
:10002000002EFED70000EF2EF2D762EF00F0010E97
:10003000055E0CE3EA6A050EE96EEF5007E0020E7A
:10004000006E002EFED700D0EF2EF9D77FEF00F024
:10005000F86AD09EEA6AE96AC150C00B0F09C16E06
:10006000070EB46EC150C00B0F09C16EC090C09294
:10007000C094C09EC2809698C69A949E9380939294
:10008000010EC66E000EC76ED190800ED56ECD6A81
:10009000000ECA6E000ECB6EB16A9484BD6AB76A58
:1000A000B66A070EB46E9250926E270E006E002E46
:1000B000FED700D0B450A19CB56A040E956E320EE6
:1000C000056EA0D78C988C9A8C9E928880A80CD0B4
:1000D00083ACFED78C888C8E8C8A8C988C9E8C9A64
:1000E0008C8E8C8A8C9E8C9A928880B818D08C8E3C
:1000F00083ACFED78C888C98960E056E98D78C8A28
:100100008C9A030E006E002EFED700D08C8A8C9A3B
:10011000270E006E002EFED700D08C8A8C9ACFD787
:020120000300DA
:020000040030CA
:0E00000024CE390E0087A1000FC00FE00F4084
:00000001FF
